 gles1test1

 Timestamp is 4be8cfea (Tue May 11 12:32:58 2010)

 Preferred load address is 00010000

 Start         Length     Name                   Class
 0001:00000000 00000004H .CRT$XCA                CODE
 0001:00000004 00000004H .CRT$XCZ                CODE
 0001:00000008 00000004H .CRT$XIA                CODE
 0001:0000000c 00000004H .CRT$XIZ                CODE
 0001:00000010 00000004H .CRT$XPA                CODE
 0001:00000014 00000004H .CRT$XPZ                CODE
 0001:00000018 00000004H .CRT$XTA                CODE
 0001:0000001c 00000004H .CRT$XTZ                CODE
 0001:00000020 000004a4H .rdata                  CODE
 0001:000004c4 00000027H .rdata$debug            CODE
 0001:000004ec 00001180H .text                   CODE
 0001:0000166c 00000014H .xdata                  CODE
 0001:00001680 00000028H .idata$2                CODE
 0001:000016a8 00000014H .idata$3                CODE
 0001:000016bc 00000110H .idata$4                CODE
 0001:000017cc 0000001cH .idata$6                CODE
 0001:000017e8 00000000H .edata                  CODE
 0002:00000000 00000110H .idata$5                DATA
 0002:00000110 000000d8H .data                   DATA
 0002:000001e8 00004024H .bss                    DATA
 0003:00000000 00000080H .pdata                  DATA

  Address         Publics by Value              Rva+Base       Lib:Object

 0000:00000000       ___safe_se_handler_count   00000000     <absolute>
 0000:00000000       ___safe_se_handler_table   00000000     <absolute>
 0001:00000000       __xc_a                     00011000     corelib0:crt0init.obj
 0001:00000004       __xc_z                     00011004     corelib0:crt0init.obj
 0001:00000008       __xi_a                     00011008     corelib0:crt0init.obj
 0001:0000000c       __xi_z                     0001100c     corelib0:crt0init.obj
 0001:00000010       __xp_a                     00011010     corelib0:crt0init.obj
 0001:00000014       __xp_z                     00011014     corelib0:crt0init.obj
 0001:00000018       __xt_a                     00011018     corelib0:crt0init.obj
 0001:0000001c       __xt_z                     0001101c     corelib0:crt0init.obj
 0001:0000003c       ??_C@_0BA@ECMACICF@EGL_BAD_SURFACE?$AA@ 0001103c     gles1test1.obj
 0001:0000004c       ??_C@_0BC@OMABNJPB@EGL_BAD_PARAMETER?$AA@ 0001104c     gles1test1.obj
 0001:00000060       ??_C@_0BG@JCAPPMPM@EGL_BAD_NATIVE_WINDOW?$AA@ 00011060     gles1test1.obj
 0001:00000078       ??_C@_0BG@IANPFEBH@EGL_BAD_NATIVE_PIXMAP?$AA@ 00011078     gles1test1.obj
 0001:00000090       ??_C@_0O@GCFMIHO@EGL_BAD_MATCH?$AA@ 00011090     gles1test1.obj
 0001:000000a0       ??_C@_0BA@KHKFAGME@EGL_BAD_DISPLAY?$AA@ 000110a0     gles1test1.obj
 0001:000000b0       ??_C@_0BI@KBFIGPCO@EGL_BAD_CURRENT_SURFACE?$AA@ 000110b0     gles1test1.obj
 0001:000000c8       ??_C@_0BA@FPCJCEFK@EGL_BAD_CONTEXT?$AA@ 000110c8     gles1test1.obj
 0001:000000d8       ??_C@_0P@HOPKKPDK@EGL_BAD_CONFIG?$AA@ 000110d8     gles1test1.obj
 0001:000000e8       ??_C@_0BC@NLAJAPHP@EGL_BAD_ATTRIBUTE?$AA@ 000110e8     gles1test1.obj
 0001:000000fc       ??_C@_0O@PGDEJDGL@EGL_BAD_ALLOC?$AA@ 000110fc     gles1test1.obj
 0001:0000010c       ??_C@_0P@ELJNOEME@EGL_BAD_ACCESS?$AA@ 0001110c     gles1test1.obj
 0001:0000011c       ??_C@_0BE@JIJLFFAN@EGL_NOT_INITIALIZED?$AA@ 0001111c     gles1test1.obj
 0001:00000130       ??_C@_0M@JFIJMCIK@EGL_SUCCESS?$AA@ 00011130     gles1test1.obj
 0001:00000174       ??_C@_0CF@GLNKALBC@?8?$CFs?8?5returned?5egl?5error?5?8?$CFs?8?5?$CI0x@ 00011174     gles1test1.obj
 0001:0000019c       ??_C@_0DG@HMPOADHB@?9?9?9?9?9?9?9?9?9?9?9?9?9?9?9?9?9?9?9?9?9?5finished?5?9@ 0001119c     gles1test1.obj
 0001:000001d4       ??_C@_0P@PNPBPNLI@eglMakeCurrent?$AA@ 000111d4     gles1test1.obj
 0001:000001e4       ??_C@_0BB@KEKMNHDF@eglCreateContext?$AA@ 000111e4     gles1test1.obj
 0001:000001f8       ??_C@_0BH@MDMCFBDG@eglCreateWindowSurface?$AA@ 000111f8     gles1test1.obj
 0001:00000210       ??_C@_0BA@GKADIFMO@eglChooseConfig?$AA@ 00011210     gles1test1.obj
 0001:00000220       ??_C@_0O@OMNEJBKO@eglGetConfigs?$AA@ 00011220     gles1test1.obj
 0001:00000230       ??_C@_0O@EEJFKEKH@eglInitialize?$AA@ 00011230     gles1test1.obj
 0001:00000240       ??_C@_0DF@DFKFEDON@?9?9?9?9?9?9?9?9?9?9?9?9?9?9?9?9?9?9?9?9?9?5started?5?9?9@ 00011240     gles1test1.obj
 0001:00000278       ??_C@_1EI@KHNCANBJ@?$AAF?$AAa?$AAi?$AAl?$AAe?$AAd?$AA?5?$AAt?$AAo?$AA?5?$AAc?$AAr?$AAe?$AAa?$AAt?$AAe?$AA?5?$AAt?$AAh?$AAe?$AA?5?$AAd?$AAe?$AAv?$AAi?$AAc?$AAe?$AA?5?$AAc?$AAo?$AAn?$AAt@ 00011278     wince_unittests.obj
 0001:000002c0       ??_C@_1BO@KHIAJBLA@?$AAI?$AAn?$AAi?$AAt?$AAi?$AAa?$AAl?$AAi?$AAz?$AAa?$AAt?$AAi?$AAo?$AAn?$AA?$AA@ 000112c0     wince_unittests.obj
 0001:000002e0       ??_C@_1EI@HEMGLDEE@?$AAF?$AAa?$AAi?$AAl?$AAe?$AAd?$AA?5?$AAt?$AAo?$AA?5?$AAr?$AAe?$AAg?$AAi?$AAs?$AAt?$AAe?$AAr?$AA?5?$AAt?$AAh?$AAe?$AA?5?$AAw?$AAi?$AAn?$AAd?$AAo?$AAw?$AA?5?$AAc?$AAl@ 000112e0     wince_unittests.obj
 0001:00000328       ??_C@_1BM@GPEKOMLI@?$AAP?$AAV?$AAR?$AAS?$AAh?$AAe?$AAl?$AAl?$AAC?$AAl?$AAa?$AAs?$AAs?$AA?$AA@ 00011328     wince_unittests.obj
 0001:00000344       ??_C@_07CHIKDHJG@?9height?$AA@ 00011344     wince_unittests.obj
 0001:0000034c       ??_C@_06EGEBBOP@?9width?$AA@ 0001134c     wince_unittests.obj
 0001:00000354       ??_C@_05MHNCFLJI@?9posy?$AA@ 00011354     wince_unittests.obj
 0001:0000035c       ??_C@_05NOMJGKNJ@?9posx?$AA@ 0001135c     wince_unittests.obj
 0001:00000368       ??_C@_1KE@BDGMONOJ@?$AAH?$AA?3?$AA?2?$AAW?$AAI?$AAN?$AAC?$AAE?$AA6?$AA0?$AA0?$AA?2?$AAP?$AAL?$AAA?$AAT?$AAF?$AAO?$AAR?$AAM?$AA?2?$AAS?$AAM?$AAD?$AAK?$AAV?$AA2?$AA1?$AA0?$AA?2?$AAS?$AAR@ 00011368     wince_unittests.obj
 0001:0000040c       ??_C@_1CI@OHCJFJPM@?$AAE?$AAR?$AAR?$AAO?$AAR?$AA?3?$AA?5?$AA?$CF?$AAs?$AA?5?$AAl?$AAi?$AAn?$AAe?$AA?5?$AA?$CF?$AAd?$AA?3?$AA?5?$AA?$AA@ 0001140c     wince_unittests.obj
 0001:00000434       ??_C@_1CK@MPGKAOE@?$AA?$CI?$AAe?$AAr?$AAr?$AAo?$AAr?$AA?5?$AAc?$AAo?$AAd?$AAe?$AA?3?$AA?5?$AA?$CF?$AAd?$AA?$CJ?$AA?3?$AA?5?$AA?$CF?$AAs?$AA?$AA@ 00011434     wince_unittests.obj
 0001:00000460       ??_C@_1M@DMCDIEDK@?$AAP?$AAK?$AAM?$AA1?$AA?3?$AA?$AA@ 00011460     wince_unittests.obj
 0001:0000046c       ??_C@_0L@GPAGIAIC@?9disablepm?$AA@ 0001146c     wince_unittests.obj
 0001:00000478       ??_C@_1M@ILHOPKA@?$AAE?$AAr?$AAr?$AAo?$AAr?$AA?$AA@ 00011478     wince_unittests.obj
 0001:00000484       ??_C@_1DG@PCJNAHOH@?$AAF?$AAa?$AAi?$AAl?$AAe?$AAd?$AA?5?$AAt?$AAo?$AA?5?$AAg?$AAe?$AAt?$AA?5?$AAm?$AAo?$AAn?$AAi?$AAt?$AAo?$AAr?$AA?5?$AAi?$AAn?$AAf?$AAo?$AA?$AA@ 00011484     wince_unittests.obj
 0001:000004bc       ??_C@_07FBLHGNAH@app?4exe?$AA@ 000114bc     wince_unittests.obj
 0001:00000548       init                       00011548 f   gles1test1.obj
 0001:00000690       display                    00011690 f   gles1test1.obj
 0001:000007ac       main                       000117ac f   gles1test1.obj
 0001:00000ab0       AppWndProc                 00011ab0 f   wince_unittests.obj
 0001:00000b10       WinMain                    00011b10 f   wince_unittests.obj
 0001:0000104c       glTexParameterf            0001204c f   libGLES_CM:libGLES_CM.dll
 0001:0000105c       glTexImage2D               0001205c f   libGLES_CM:libGLES_CM.dll
 0001:0000106c       glTexCoordPointer          0001206c f   libGLES_CM:libGLES_CM.dll
 0001:0000107c       glColorPointer             0001207c f   libGLES_CM:libGLES_CM.dll
 0001:0000108c       glVertexPointer            0001208c f   libGLES_CM:libGLES_CM.dll
 0001:0000109c       glEnableClientState        0001209c f   libGLES_CM:libGLES_CM.dll
 0001:000010ac       glShadeModel               000120ac f   libGLES_CM:libGLES_CM.dll
 0001:000010bc       glClearColor               000120bc f   libGLES_CM:libGLES_CM.dll
 0001:000010cc       glDisable                  000120cc f   libGLES_CM:libGLES_CM.dll
 0001:000010dc       glDrawArrays               000120dc f   libGLES_CM:libGLES_CM.dll
 0001:000010ec       glEnable                   000120ec f   libGLES_CM:libGLES_CM.dll
 0001:000010fc       glRotatef                  000120fc f   libGLES_CM:libGLES_CM.dll
 0001:0000110c       glTranslatef               0001210c f   libGLES_CM:libGLES_CM.dll
 0001:0000111c       glLoadIdentity             0001211c f   libGLES_CM:libGLES_CM.dll
 0001:0000112c       glMatrixMode               0001212c f   libGLES_CM:libGLES_CM.dll
 0001:0000113c       glClear                    0001213c f   libGLES_CM:libGLES_CM.dll
 0001:0000114c       GetDC                      0001214c f   coredll:COREDLL.dll
 0001:0000115c       PostQuitMessage            0001215c f   coredll:COREDLL.dll
 0001:0000116c       DefWindowProcW             0001216c f   coredll:COREDLL.dll
 0001:0000117c       ReleasePowerRequirement    0001217c f   coredll:COREDLL.dll
 0001:0000118c       DestroyWindow              0001218c f   coredll:COREDLL.dll
 0001:0000119c       ReleaseDC                  0001219c f   coredll:COREDLL.dll
 0001:000011ac       CreateWindowExW            000121ac f   coredll:COREDLL.dll
 0001:000011bc       RegisterClassW             000121bc f   coredll:COREDLL.dll
 0001:000011cc       GetStockObject             000121cc f   coredll:COREDLL.dll
 0001:000011dc       NKDbgPrintfW               000121dc f   coredll:COREDLL.dll
 0001:000011ec       FormatMessageW             000121ec f   coredll:COREDLL.dll
 0001:000011fc       GetLastError               000121fc f   coredll:COREDLL.dll
 0001:0000120c       SetPowerRequirement        0001220c f   coredll:COREDLL.dll
 0001:0000121c       WideCharToMultiByte        0001221c f   coredll:COREDLL.dll
 0001:0000122c       SetCursorPos               0001222c f   coredll:COREDLL.dll
 0001:0000123c       GetCursorPos               0001223c f   coredll:COREDLL.dll
 0001:0000124c       MessageBoxW                0001224c f   coredll:COREDLL.dll
 0001:0000125c       GetMonitorInfo             0001225c f   coredll:COREDLL.dll
 0001:0000126c       MonitorFromPoint           0001226c f   coredll:COREDLL.dll
 0001:0000127c       GetSystemMetrics           0001227c f   coredll:COREDLL.dll
 0001:0000130c       WinMainCRTStartup          0001230c f   corelib0:pegwmain.obj
 0001:00001408       exit                       00012408 f   corelib0:cexit.obj
 0001:00001420       _exit                      00012420 f   corelib0:cexit.obj
 0001:00001460       __security_init_cookie     00012460 f   corelib0:seccinit.obj
 0001:000014bc       __security_check_cookie    000124bc f   corelib0:armsecgs.obj
 0001:000014d0       __gsfailure                000124d0 f   corelib0:armsecgs.obj
 0001:00001514       _initterm                  00012514 f   corelib0:crt0dat.obj
 0001:00001548       _cinit                     00012548 f   corelib0:crt0dat.obj
 0001:0000157c       fprintf                    0001257c f   corelib1:COREDLL.dll
 0001:0000158c       _getstdfilex               0001258c f   corelib1:COREDLL.dll
 0001:0000159c       atol                       0001259c f   corelib1:COREDLL.dll
 0001:000015ac       atoi                       000125ac f   corelib1:COREDLL.dll
 0001:000015bc       _stricmp                   000125bc f   corelib1:COREDLL.dll
 0001:000015cc       _isctype                   000125cc f   corelib1:COREDLL.dll
 0001:000015dc       malloc                     000125dc f   corelib1:COREDLL.dll
 0001:000015ec       wcslen                     000125ec f   corelib1:COREDLL.dll
 0001:000015fc       memset                     000125fc f   corelib1:COREDLL.dll
 0001:0000160c       _XcptFilter                0001260c f   corelib1:COREDLL.dll
 0001:0000161c       __C_specific_handler       0001261c f   corelib1:COREDLL.dll
 0001:0000162c       free                       0001262c f   corelib1:COREDLL.dll
 0001:0000163c       __security_gen_cookie2     0001263c f   corelib1:COREDLL.dll
 0001:0000164c       __report_gsfailure         0001264c f   corelib1:COREDLL.dll
 0001:0000165c       TerminateProcess           0001265c f   coredll:COREDLL.dll
 0001:00001680       __IMPORT_DESCRIPTOR_libGLES_CM 00012680     libGLES_CM:libGLES_CM.dll
 0001:00001694       __IMPORT_DESCRIPTOR_COREDLL 00012694     coredll:COREDLL.dll
 0001:000016a8       __NULL_IMPORT_DESCRIPTOR   000126a8     libGLES_CM:libGLES_CM.dll
 0002:00000000       __imp_DestroyWindow        00013000     coredll:COREDLL.dll
 0002:00000004       __imp___report_gsfailure   00013004     corelib1:COREDLL.dll
 0002:00000008       __imp___security_gen_cookie2 00013008     corelib1:COREDLL.dll
 0002:0000000c       __imp_free                 0001300c     corelib1:COREDLL.dll
 0002:00000010       __imp___C_specific_handler 00013010     corelib1:COREDLL.dll
 0002:00000014       __imp__XcptFilter          00013014     corelib1:COREDLL.dll
 0002:00000018       __imp_memset               00013018     corelib1:COREDLL.dll
 0002:0000001c       __imp_wcslen               0001301c     corelib1:COREDLL.dll
 0002:00000020       __imp_malloc               00013020     corelib1:COREDLL.dll
 0002:00000024       __imp__isctype             00013024     corelib1:COREDLL.dll
 0002:00000028       __imp__stricmp             00013028     corelib1:COREDLL.dll
 0002:0000002c       __imp_atoi                 0001302c     corelib1:COREDLL.dll
 0002:00000030       __imp_atol                 00013030     corelib1:COREDLL.dll
 0002:00000034       __imp___muls               00013034     corelib1:COREDLL.dll
 0002:00000038       __imp___itos               00013038     corelib1:COREDLL.dll
 0002:0000003c       __imp__getstdfilex         0001303c     corelib1:COREDLL.dll
 0002:00000040       __imp_fprintf              00013040     corelib1:COREDLL.dll
 0002:00000044       __imp_GetSystemMetrics     00013044     coredll:COREDLL.dll
 0002:00000048       __imp_MonitorFromPoint     00013048     coredll:COREDLL.dll
 0002:0000004c       __imp_GetMonitorInfo       0001304c     coredll:COREDLL.dll
 0002:00000050       __imp_MessageBoxW          00013050     coredll:COREDLL.dll
 0002:00000054       __imp_GetCursorPos         00013054     coredll:COREDLL.dll
 0002:00000058       __imp_SetCursorPos         00013058     coredll:COREDLL.dll
 0002:0000005c       __imp_WideCharToMultiByte  0001305c     coredll:COREDLL.dll
 0002:00000060       __imp_SetPowerRequirement  00013060     coredll:COREDLL.dll
 0002:00000064       __imp_GetLastError         00013064     coredll:COREDLL.dll
 0002:00000068       __imp_GetDC                00013068     coredll:COREDLL.dll
 0002:0000006c       __imp_PostQuitMessage      0001306c     coredll:COREDLL.dll
 0002:00000070       __imp_DefWindowProcW       00013070     coredll:COREDLL.dll
 0002:00000074       __imp_ReleasePowerRequirement 00013074     coredll:COREDLL.dll
 0002:00000078       __imp_TerminateProcess     00013078     coredll:COREDLL.dll
 0002:0000007c       __imp_ReleaseDC            0001307c     coredll:COREDLL.dll
 0002:00000080       __imp_CreateWindowExW      00013080     coredll:COREDLL.dll
 0002:00000084       __imp_RegisterClassW       00013084     coredll:COREDLL.dll
 0002:00000088       __imp_GetStockObject       00013088     coredll:COREDLL.dll
 0002:0000008c       __imp_NKDbgPrintfW         0001308c     coredll:COREDLL.dll
 0002:00000090       __imp_FormatMessageW       00013090     coredll:COREDLL.dll
 0002:00000094       \177COREDLL_NULL_THUNK_DATA 00013094     coredll:COREDLL.dll
 0002:00000098       __imp_eglInitialize        00013098     libGLES_CM:libGLES_CM.dll
 0002:0000009c       __imp_eglGetDisplay        0001309c     libGLES_CM:libGLES_CM.dll
 0002:000000a0       __imp_eglGetConfigs        000130a0     libGLES_CM:libGLES_CM.dll
 0002:000000a4       __imp_eglChooseConfig      000130a4     libGLES_CM:libGLES_CM.dll
 0002:000000a8       __imp_eglCreateWindowSurface 000130a8     libGLES_CM:libGLES_CM.dll
 0002:000000ac       __imp_eglCreateContext     000130ac     libGLES_CM:libGLES_CM.dll
 0002:000000b0       __imp_eglMakeCurrent       000130b0     libGLES_CM:libGLES_CM.dll
 0002:000000b4       __imp_eglSwapInterval      000130b4     libGLES_CM:libGLES_CM.dll
 0002:000000b8       __imp_eglSwapBuffers       000130b8     libGLES_CM:libGLES_CM.dll
 0002:000000bc       __imp_eglTerminate         000130bc     libGLES_CM:libGLES_CM.dll
 0002:000000c0       __imp_eglDestroySurface    000130c0     libGLES_CM:libGLES_CM.dll
 0002:000000c4       __imp_eglDestroyContext    000130c4     libGLES_CM:libGLES_CM.dll
 0002:000000c8       __imp_glClear              000130c8     libGLES_CM:libGLES_CM.dll
 0002:000000cc       __imp_glMatrixMode         000130cc     libGLES_CM:libGLES_CM.dll
 0002:000000d0       __imp_glLoadIdentity       000130d0     libGLES_CM:libGLES_CM.dll
 0002:000000d4       __imp_glTranslatef         000130d4     libGLES_CM:libGLES_CM.dll
 0002:000000d8       __imp_glRotatef            000130d8     libGLES_CM:libGLES_CM.dll
 0002:000000dc       __imp_glEnable             000130dc     libGLES_CM:libGLES_CM.dll
 0002:000000e0       __imp_glDrawArrays         000130e0     libGLES_CM:libGLES_CM.dll
 0002:000000e4       __imp_glDisable            000130e4     libGLES_CM:libGLES_CM.dll
 0002:000000e8       __imp_glClearColor         000130e8     libGLES_CM:libGLES_CM.dll
 0002:000000ec       __imp_glShadeModel         000130ec     libGLES_CM:libGLES_CM.dll
 0002:000000f0       __imp_glEnableClientState  000130f0     libGLES_CM:libGLES_CM.dll
 0002:000000f4       __imp_glVertexPointer      000130f4     libGLES_CM:libGLES_CM.dll
 0002:000000f8       __imp_glColorPointer       000130f8     libGLES_CM:libGLES_CM.dll
 0002:000000fc       __imp_glTexCoordPointer    000130fc     libGLES_CM:libGLES_CM.dll
 0002:00000100       __imp_glTexImage2D         00013100     libGLES_CM:libGLES_CM.dll
 0002:00000104       __imp_glTexParameterf      00013104     libGLES_CM:libGLES_CM.dll
 0002:00000108       __imp_eglGetError          00013108     libGLES_CM:libGLES_CM.dll
 0002:0000010c       \177libGLES_CM_NULL_THUNK_DATA 0001310c     libGLES_CM:libGLES_CM.dll
 0002:000001d0       gui32WindowWidth           000131d0     wince_unittests.obj
 0002:000001d4       gui32WindowHeight          000131d4     wince_unittests.obj
 0002:000001d8       gui32PosX                  000131d8     wince_unittests.obj
 0002:000001dc       gui32PosY                  000131dc     wince_unittests.obj
 0002:000001e0       __security_cookie          000131e0     corelib0:seccinit.obj
 0002:000001e4       __security_cookie_complement 000131e4     corelib0:seccinit.obj
 0002:000041ec       gbWindow                   000171ec     wince_unittests.obj
 0002:000041f0       ghWnd                      000171f0     wince_unittests.obj
 0002:000041f4       pfnRegisteredWndProc       000171f4     wince_unittests.obj
 0002:000041f8       _exitflag                  000171f8     corelib0:cexit.obj
 0002:000041fc       gui32DisplayWidth          000171fc     <common>
 0002:00004200       gui32DisplayHeight         00017200     <common>
 0002:00004204       __onexitend                00017204     <common>
 0002:00004208       __onexitbegin              00017208     <common>

 entry point at        0001:0000130c

 Static symbols

 0001:000004ec       handle_egl_error           000114ec f   gles1test1.obj
 0001:00001294       WinMainCRTStartupHelper    00012294 f   corelib0:pegwmain.obj
 0001:00001340       doexit                     00012340 f   corelib0:cexit.obj
